S00E00007365726D75782E7372656372
S113000019C033C032C031C030C02FC02EC02DC083
S11300102CC02BC02AC029C028C027C026C025C098
S113002025C023C022C021C020C01FC01EC01DC0C7
S11300301CC01BC011241FBECFEFD4E0DEBFCDBF58
S113004011E0A0E0B1E0EEE6F3E002C005900D920D
S1130050A030B107D9F714E0A0E0B1E001C01D92CF
S1130060A130B107E1F785D081C1CACF8FB68F9295
S1130070FA947AF403E0F02E00911401E02FFF27A4
S1130080E050FF4F01500AF403E100931401908003
S113009095B886B0880C880C06E0E0E5F2E009C06B
S11300A09180880C97949182139510830A9562F13C
S11300B0E05110811B3149F01034A4F410321AF0CD
S11300C0212F237069F3880CEFCF880C68F7248103
S11300D0203C61F728830983CE5FC0930004222764
S11300E02483E4CF880C70F0203451F424812074EC
S11300F02483202B288321812983CE5FC09300048D
S11301001BE1D3CF1CE1D1CFF091C000F07269F0B4
S1130110F0910004E0916002FE1739F0F3E0808072
S11301208092C600E395E0936002F091C000F078FD
S1130130E9F00091C600E0916102EF3F31F406302E
S113014008F006E00093610211C0E63060F4F2E0CA
S1130150E2951281E10F008313951770E07F1283FB
S11301601481106414830FEF009361028F908FBE8B
S11301701895F894CFEFD4E0DEBFCDBF8FE384B9F8
S113018003E004BD0BE005BD05E007BD02E00093FC
S11301906E000FE00093C40002E00093C00008E189
S11301A00093C10006E00093C20006E01BE120E0DA
S11301B0E0E0F2E01083248322832383E05F0A9546
S11301C0C9F7A0E0B3E094E18FEF8C93A3959A95DF
S11301D0E1F793E190931401FF24CC27D3E0C0937B
S11301E00004C093600299E0789480911401891707
S11301F0E1F79A500AF493E1B2E000240A94102C37
S1130200202C302C402C502C6FEFE894709102027B
S113021080910302781751F08A2FA85F0C90839580
S113022087708093030260F9781749F4F894709109
S11302300402872F880F782B7093040278947091AE
S1130240120280911302781751F08A2FA85E1C9035
S1130250839587708093130261F9781749F4F894B1
S113026070911402872F880F782B7093140278945E
S11302707091220280912302781751F08A2FA85D91
S11302802C90839587708093230262F9781749F440
S1130290F89470912402872F880F782B709324028E
S11302A078947091320280913302781751F08A2F3A
S11302B0A85C3C90839587708093330263F9781728
S11302C049F4F89470913402872F880F782B709337
S11302D0340278947091420280914302781751F06D
S11302E08A2FA85B4C90839587708093430264F9AE
S11302F0781749F4F89470914402872F880F782B6B
S1130300709344027894709152028091530278174A
S113031051F08A2FA85A5C9083958770809353027A
S113032065F9781749F4F89470915402872F880F6F
S1130330782B709354027894A0E0B1E0A90F88E080
S11303406C93AA956FEF5694661F4694661F369475
S1130350661F2694661F1694661F0694661F6C9388
S1110360AA958A9579F76FEF6C933FCFFFCF84
S9030000FC
